:020000040000FA
:0400000025EF00F0F8
:0200080037D0EF
:0800180085D0046A036EFF0E9F
:100020000326042200D0D8A01200030E026EE70EB1
:1000300002D8F5D7026AFE0F016EE86A025AD8A00C
:1000400012000000010600D0F8D7F86A4F0EAF6E1C
:10005000240EAC6E900EAB6E0001070EB46E0F0E48
:10006000C16EC69AC00E926EE00E936EC00E946E74
:10007000956AE80E966EE6D09EAA1BD0060EAB14CB
:1000800012E1E1CF2BF0E2CF2CF02D2A1EEE80F012
:100090002D50E126000EE222AECFE7FF2BC0E1FF9C
:1000A0002CC0E2FF1100AE50AE50AB98AB881100EF
:1000B0000AD0F2A408D0F294074A082A817A066A84
:1000C000D6CF05F0110011002D502E5C14E02E2A21
:1000D000E9CF01F0EACF02F00EEE80F02E50E926D3
:1000E000000EEA22EF50016E01C0E9FF02C0EAFFF4
:1000F000D880120004D0E868016ED8A01200120067
:100100002D6A2E6A9D8A9F8AF28EF28C12009D9A29
:100110000EEE80F0000EEE6AE82EFDD72D6A2E6AF4
:100120009D8A1200F29ED8CF59FEE8CF5AFEE0CF4A
:100130005BFEE9CF5CFEEACF5DFEE1CF5EFEE2CF83
:100140005FFED9CF60FEDACF61FEF6CF62FEF7CF59
:1001500063FEF5CF64FEF3CF65FEF4CF66FEA6CF57
:1001600067FE01C068FEF28E0001A1921FA228D096
:1001700025C0B2FF26C0B3FF0B4A0C2A0BA21FD02A
:100180000B6A0C6A2F50016E0C0819E3FA6A0136EB
:10019000FA36A40E0126010EFA22FB6A000EFB229B
:1001A0000150F96E28D00FD010D011D012D013D03A
:1001B00014D015D016D017D018D019D01AD01BD003
:1001C0000B6A0C6A18D0837216D0827614D08272B1
:1001D00012D0837410D082780ED083780CD0837CB8
:1001E0000AD0817008D0817406D0817804D08472DE
:1001F00002D0807A00D0F29E59CED8FF5ACEE8FFC6
:100200005BCEE0FF5CCEE9FF5DCEEAFF5ECEE1FFB4
:100210005FCEE2FF60CED9FF61CEDAFF62CEF6FF9D
:1002200063CEF7FF64CEF5FF65CEF3FF66CEF4FF35
:1002300067CEA6FF68CE01F0F28E10009EA8FED712
:10024000AD6E1200939A8A8A0A0EE7DE939A8A9A12
:10025000F3EC04F030EC05F0206A780E226E0A0E02
:10026000286E22C024F0236AD890243628C02AF0B1
:10027000296AD8902A36276A43DF49DFCD6AF2948B
:10028000F28A870ED56EB16AA192A082B26AB36A71
:10029000D08EA292B10EB16E17DF0D6EBB0E0D5C4B
:1002A00005E3FE0E0D5C01E20E6AF0D10DAE20D02A
:1002B0000E6A8A0E0D5C05E10DC00EF00F68106825
:1002C00016D09A0E0D5C05E10DC00EF01168126893
:1002D0000ED0BA0E0D5C05E10DC00EF01368146867
:1002E00006D0DA0E0D5C03E10DC00EF01668CED11B
:1002F0000E5202E1CBD1CAD18A0E0E5CD8A46FD0C7
:100300000F2803E10DC00FF068D00DC010F0270ECC
:100310000F5CD8A061D0580E0F5CD8B05DD0270E0E
:100320000F5C00EE31F0EB50006E305CD8A451D081
:100330003052D8B44AD03050016E0C0831E3FA6A1A
:10034000D8900136FA360136FA366C0E0126030EC5
:10035000FA22FB6A000EFB220500FF6A000EFF2254
:10036000030EFE6EA00EFD6E0150F96E79EF04F0E3
:100370007AEF04F07CEF04F07EEF04F080EF04F0FD
:1003800082EF04F084EF04F086EF04F088EF04F0CD
:100390008AEF04F08CEF04F08EEF04F090EF04F09D
:1003A000B1901F921F94D6CF05F0D7CF06F02350FF
:1003B0000524176E24500620186E000E0720196EB3
:1003C000000E08201A6E1F8003D01F901F921F94EA
:1003D00003D01F901F921F940F6858D157D19A0EC7
:1003E0000E5CD8A43FD1112803E10DC011F039D122
:1003F0000DC012F01252D8A466D0270E115CD8A0FE
:1004000061D0580E115CD8B05DD0270E115C00EEA3
:1004100031F0EB50006E305CD8A451D03052D8B4DB
:100420004AD03050016E0C0831E3FA6AD890013698
:10043000FA360136FA36580E0126040EFA22FB6A05
:10044000000EFB220500FF6A000EFF22040EFE6E66
:100450008C0EFD6E0150F96E79EF04F07AEF04F026
:100460007CEF04F07EEF04F080EF04F082EF04F004
:1004700084EF04F086EF04F088EF04F08AEF04F0D4
:100480008CEF04F08EEF04F090EF04F0B1901F9227
:100490001F94D6CF05F0D7CF06F023500524176E52
:1004A00024500620186E000E0720196E000E08203A
:1004B0001A6E1F8003D01F901F921F9403D01F90AD
:1004C0001F921F94CED0270E115CD8A0C9D0580E11
:1004D000115CD8B0C5D0270E115C216E00EE31F052
:1004E0002150EB502F6E2F50305CD8B47FD01F922C
:1004F0002F50016E0C0831E3FA6AD8900136FA36B3
:100500000136FA36260E0126050EFA22FB6A000E87
:10051000FB220500FF6A000EFF22050EFE6E5A0E3A
:10052000FD6E0150F96E22EF04F023EF04F026EF88
:1005300004F029EF04F02CEF04F02FEF04F032EF79
:1005400004F035EF04F038EF04F03BEF04F03EEF39
:1005500004F041EF04F044EF04F0D6CF05F0D7CF1C
:1005600006F0295005241B6E2A5006201C6E000E32
:1005700007201D6E000E08201E6E1F843050016E75
:100580000C0831E3FA6AD8900136FA360136FA36A9
:10059000B20E0126050EFA22FB6A000EFB220500B0
:1005A000FF6A000EFF22050EFE6EE60EFD6E015084
:1005B000F96EFDEF03F0FEEF03F001EF04F004EF3E
:1005C00004F007EF04F00AEF04F00DEF04F010EF71
:1005D00004F013EF04F016EF04F019EF04F01CEF31
:1005E00004F01FEF04F02FC030F039D02F50016E0F
:1005F0000C0831E3FA6AD8900136FA360136FA3639
:10060000220E0126060EFA22FB6A000EFB220500CE
:10061000FF6A000EFF22060EFE6E560EFD6E0150A2
:10062000F96E47EF04F048EF04F04AEF04F04CEFA6
:1006300004F04EEF04F050EF04F052EF04F054EFEA
:1006400004F056EF04F058EF04F05AEF04F05CEFBA
:1006500004F05EEF04F0275202E01F82B1801F9089
:10066000116814D0BA0E0E5C09E1132803E10DC025
:1006700013F003D00DC014F06BD908D0DA0E0E5C65
:1006800005E1162803E10DC016F04CD91FA049D092
:10069000D6CF05F0D7CF06F01750055C1850065896
:1006A000195007581A50085808501A18D8B0800A1C
:1006B00038E73050016E0C0831E3FA6AD890013601
:1006C000FA360136FA36E80E0126060EFA22FB6AE1
:1006D000000EFB220500FF6A000EFF22070EFE6ED1
:1006E0001C0EFD6E0150F96EFDEF03F0FEEF03F0FE
:1006F00001EF04F004EF04F007EF04F00AEF04F058
:100700000DEF04F010EF04F013EF04F016EF04F017
:1007100019EF04F01CEF04F01FEF04F02F6A306AA9
:100720001F901FA44ED0D6CF05F0D7CF06F01B5098
:10073000055C1C5006581D5007581E50085808509C
:100740001E18D8B0800A3DE72F50016E0C0831E327
:10075000FA6AD8900136FA360136FA367E0E01264C
:10076000070EFA22FB6A000EFB220500FF6A000E4C
:10077000FF22070EFE6EB20EFD6E0150F96E79EF8C
:1007800004F07AEF04F07CEF04F07EEF04F080EFE9
:1007900004F082EF04F084EF04F086EF04F088EFB9
:1007A00004F08AEF04F08CEF04F08EEF04F090EF89
:1007B00004F0275203E01F82B18002D01F92B19053
:1007C0001F944CEF01F0306A12008C9012008B9451
:1007D00012008B9012008C9612008B9A12008C9A49
:1007E00012008C9E12008A9212008A9612008D943A
:1007F00012008D9012008998120012008C908C9239
:1008000012008B948B9612008B908B9212008C9618
:100810008C9412008B9A8B9812008C9A8C981200F0
:100820008C9E8C9C12008A928A9012008A968A94DE
:1008300012008D948A9812008D908D9212008998E2
:10084000899A120012008C828C8012008B868B8415
:1008500012008B828B8012008C848C8612008B8815
:100860008B8A12008C888C8A12008C8C8C8E1200E1
:100870008A808A8212008A848A8612008A888D84FD
:1008800012008D828D801200898A898812001200E0
:100890008C8012008B8412008B8012008C861200D8
:1008A0008B8A12008C8A12008C8E12008A821200AF
:1008B0008A8612008D8412008D80120089881200B1
:1008C00012008C8212008B8612008B8212008C84A4
:1008D00012008B8812008C8812008C8C12008A8087
:1008E00012008A8412008A8812008D821200898A7E
:1008F000120012008C9212008B9612008B92120042
:100900008C9412008B9812008C9812008C9C120010
:100910008A9012008A9412008A9812008D92120016
:10092000899A120016520EE0B19016C027F027C027
:1009300026F0256AD890263625C0B2FF26C0B3FF20
:10094000B18004D0276A256A266AB1901668120021
:100950001E0E135C0EE114C022F0225204E11F901F
:10096000236A246A05D022C024F0236AD890243652
:1009700038D01F0E135C19E11450275C15E0145297
:100980000EE0B19014C027F027C026F0256AD89059
:10099000263625C0B2FF26C0B3FFB18005D0B19086
:1009A000276A256A266A1F921CD0200E135C0BE171
:1009B0001450285C07E014C028F028C02AF0296AE7
:1009C000D8902A360ED0420E135C07E1145203E190
:1009D000209009D801D0208004D07B0E135CD8B4BD
:1009E00002D8136812001F6A076A086A8C928B96F5
:1009F0008B928C948B988C988C9C8A908A948A98F1
:100A00008D92899A899689928C908B948B908C96F2
:100A10008B9A8C9A8C9E8A928A968D948D908998C6
:100A2000899089942F6A306A12008C928B968B92EF
:100A30008C948B988C988C9C8A908A948A988D92AE
:100A4000899A8C908B948B908C968B9A8C9A8C9E96
:100A50008A928A968D948D9089982F6A306A1200B6
:100A6000316A010E326E020E336E030E346E040EC6
:100A7000356E050E366E060E376E070E386E080E92
:100A8000396E090E3A6E0A0E3B6E0B0E3C6E0C0E62
:100A90003D6E010E3E6E020E3F6E030E406E040E62
:100AA000416E050E426E060E436E070E446E080E32
:100AB000456E090E466E0A0E476E0B0E486E0C0E02
:100AC000496E010E4A6E020E4B6E030E4C6E040E02
:100AD0004D6E050E4E6E060E4F6E070E506E080ED2
:100AE000516E090E526E0A0E536E0B0E546E0C0EA2
:100AF000556E010E566E020E576E030E586E040EA2
:100B0000596E050E5A6E060E5B6E070E5C6E080E71
:100B10005D6E090E5E6E0A0E5F6E0B0E606E0C0E41
:060B2000616E1200FFD718
:020000040030CA
:0300010006160ED2
:020005008580F4
:060008000FC00FE00F40E5
:00000001FF
